:103DB9000FC30FBF0FBB0FB60FB20FAC0FA70FA1E9
:103DC9000F9B0F950F8E0F870F800F780F700F685D
:103DD9000F5F0F550F4B0F410F360F2B0F1F0F1290
:103DE9000F060EF80EEA0EDB0ECC0EBC0EAB0E9AC9
:103DF9000E880E750E620E4E0E390E240E0E0DF73C
:103E09000DDF0DC70DAE0D940D790D5E0D410D241D
:103E19000D070CE80CC90CA90C890C680C460C237D
:103E29000C000BDC0BB80B930B6E0B480B210AFA39
:103E39000AD30AAC0A840A5B0A330A0A09E109B7F8
:103E4900098E0965093B091108E808BE0895086C3F
:103E59000842081907F107C807A00778075007297A
:103E6900070206DB06B5068F066A0645062105FD2B
:103E790005DA05B70595057405530532051204F3EE
:103E890004D404B60498047B045F04430428040D95
:103E990003F303DA03C103A90391037A0363034D0F
:103EA90003370322030E02F902E602D302C002AE6F
:103EB900029C028B027A026A025A024B023C022DD0
:103EC900021F0211020301F601E901DD01D001C55A
:103ED90001B901AE01A30198018E0184017A017132
:103EE9000168015F0156014D0145013D0135012E72
:103EF9000126011F01180111010B010400FE00F840
:103F090000F200EC00E600E100DC00D600D100CCB4
:103F190000C800C300BE00BA00B600010C010104CC
:103F290002011E030A960401320503030600640711
:103F3900010108000009015A0E01010F00011200D8
:103F49006413010114013C1501FA1664FA17FFFF05
:103F59001D00072000072400022701012F013C3022
:103F6900010132010335FFFF3603073CFFFF3DFF27
:103F7900FF180002191E461A00021B00022D32C842
:103F89002E0001FAFAFA18000019FFFF1A00001BA7
:103F990000002D32C82E0001FAFAFA18000019FFA4
:103FA900FF1A00001B00002DFFFF2EFFFFFAFAFA8F
:10004800900786E0FEA3E0FF7457BE0010D39F40E0
:100058000C903F2312001EE493F599804C900014F5
:10006800E0D394044014900786E0FEA3E0FF903F9D
:100078002312001EE493F599802F900014E0D39486
:10008800034014900786E0FEA3E0FF903F3812007B
:100098001EE493F5998012900786E0FEA3E0FF9096
:1000A8003F4D12001EE493F59990078612000E90BA
:1000B8000786E0FEA3E0FF746C6F4E7003751300B3
:1000C80022900072E0B402087401900072F0D20C21
:1000D80090013AE090002AF090013BE090002BF06C
:1000E80090013CE090002CF0A20AB3401690013A2F
:1000F800E0700C90013BE0700690013CE0600280EB
:1001080002C20A90013AE0B4300F90013BE0B447D4
:100118000890013CE0643B60028004D20B8002C27C
:100128000BE558B40102800302024B900057E0F53A
:1001380066900062E0F568900063E0F569900074ED
:10014800E0F56A90007AE0900029F090007CE0F5F4
:100158006590007DE0F567900080E0F5649000818F
:10016800E0F563900090E0900041F0900091E090FD
:100178000042F0900092E0900043F0900093E090ED
:100188000044F0900094E0900045F0900095E090D5
:100198000046F0900096E0900047F0900097E090BD
:1001A8000048F0900099E0900033F090009AE090B9
:1001B8000034F090009BE0900035F090009CE090B7
:1001C8000036F0900079E0B4011790000A740FF03F
:1001D800A374FFF090000CE4F0A3F074029000798F
:1001E800F0900079E0B4035990000CE0FEA3E0FF22
:1001F80090000AE0FCA3E0FD1200037410124119FC
:10020800740812410BEF900026F0EF700674FF900F
:100218000026F07400900079F090000BE090002721
:10022800F090000AE0900028F0900026E0900789FE
:10023800F0900027E090078AF0900028E090078B64
:10024800F0803F900081E07006755801756300A248
:100258000AB3402E90013AE090002AF090013BE06A
:1002680090002BF090013CE090002CF090002AE0E8
:10027800700C90002BE0700690002CE06002800269
:10028800C20AE5667003756602E568700375680260
:100298007E837FC2E5668E048F05FF1240FB8C3992
:1002A8008D3AE56975F0FAA4FFAEF0E5688E048F23
:1002B80005FF1240FB8C3D8D3E90004FE0F56090AD
:1002C800004DE0FE900069E0B5061890004CE0FE95
:1002D800900068E0B5060C90004BE0FE900059E0F5
:1002E8006E606F900069E07006900068E0600674C8
:1002F80000900059F0900069E0B402089000497439
:1003080001F08005900049E4F0900068E0B402082C
:1003180090004A7401F0800590004AE4F09000686B
:10032800E0600690004AE060028005756003800383
:10033800756004E559B55802D20C900068E0900049
:100348004CF0900069E090004DF0900059E090006A
:100358004BF0740190009EF0740190009FF07400BF
:100368009000A0F074009000A1F074009000A2F03A
:1003780074009000A3F074009000A4F07401900041
:10038800A5F074019000A6F074009000A7F0740026
:100398009000A8F074009000A9F074009000AAF0F2
:1003A80074009000ABF074019000ACF07401900000
:1003B800ADF074009000AEF074009000AFF07400DF
:1003C8009000B0F074009000B1F074009000B2F0AA
:1003D8007401900362F07401900363F07400900359
:1003E80064F07400900365F07400900366F0740084
:1003F800900367F07400900368F074009003A2F013
:1004080074019003A3F074009003A4F074009003A7
:10041800A5F074009003A6F074009003A7F0740090
:100428009003A8F074009003E2F074009003E3F0E6
:1004380074009003E4F074009003E5F074009003F6
:10044800E6F074009003E7F074009003E8F074019C
:10045800900422F07400900423F07400900424F0B7
:100468007400900425F07400900426F07400900441
:1004780027F07400900428F022E5B554F7F5B5E5A7
:10048800B554FDF5B5C2A2C2A1C292C207E5B554E2
:10049800FBF5B5755104E55104F55290004FE0F5B0
:1004A80060900025E4F0C209E5B554FEF5B5C28EAA
:1004B800758D00758B00754C00752600752500D26A
:1004C8008E22750A00750900AE09AF0A7457BE007E
:1004D800039F5003020587903F2312001EE4939068
:1004E800004E1241310FBF00010EE0FC903F231275
:1004F800001EECFEE493FFEEC39F5026AE09AF0A40
:100508000FBF00010E903F2312001EAE09AF0AE490
:1005180093FC903F2312001EE49390004E12413149
:10052800ECF0AE09AF0A903F2312001EE49390004E
:100538004E124131E0FC903F2512001EECFCE49382
:10054800FDECD39D4019903F2512001EE493FC90CA
:100558003F2312001EE49390004E124131ECF0AE9E
:1005680009AF0A74022FFF50010E8E098F0A780A0C
:10057800740126F6500418E436F640030204D0222B
:10058800750A00750900AE09AF0A7415BE00039F0D
:100598005003020655903F7A12001EE49390004ED5
:1005A8001241310FBF00010EE0FC903F7A12001E8D
:1005B800ECFEE493FFEEC39F5026AE09AF0A0FBFCF
:1005C80000010E903F7A12001EAE09AF0AE493FCB8
:1005D800903F7A12001EE49390004E124131ECF0E5
:1005E800AE09AF0A903F7A12001EE49390004E12B3
:1005F8004131E0FC903F7C12001EECFCE493FDECE2
:10060800D39D4019903F7C12001EE493FC903F7AE2
:1006180012001EE49390004E124131ECF0AE09AF87
:100628000A740F6F4E7006750A15750900AE09AF8A
:100638000A74022FFF50010E8E098F0A780A74017E
:1006480026F6500418E436F6400302058E22750A91
:1006580000750900AE09AF0A7415BE00039F500368
:10066800020723903F8F12001EE49390004E124120
:10067800310FBF00010EE0FC903F8F12001EECFE10
:10068800E493FFEEC39F5026AE09AF0A0FBF0001E7
:100698000E903F8F12001EAE09AF0AE493FC903F04
:1006A8008F12001EE49390004E124131ECF0AE0917
:1006B800AF0A903F8F12001EE49390004E12413112
:1006C800E0FC903F9112001EECFCE493FDECD39DFE
:1006D8004019903F9112001EE493FC903F8F120046
:1006E8001EE49390004E124131ECF0AE09AF0A744B
:1006F8000F6F4E7006750A15750900AE09AF0A74BA
:10070800022FFF50010E8E098F0A780A740126F60F
:10071800500418E436F6400302065C22750A007598
:100728000900AE09AF0A7415BE00039F5003020703
:10073800F1903FA412001EE49390004E1241310F35
:10074800BF00010EE0FC903FA412001EECFEE493F3
:10075800FFEEC39F5026AE09AF0A0FBF00010E90EF
:100768003FA412001EAE09AF0AE493FC903FA41206
:10077800001EE49390004E124131ECF0AE09AF0A2E
:10078800903FA412001EE49390004E124131E0FC09
:10079800903FA612001EECFCE493FDECD39D40199B
:1007A800903FA612001EE493FC903FA412001EE4A2
:1007B8009390004E124131ECF0AE09AF0A740F6FFE
:1007C8004E7006750A15750900AE09AF0A74022F36
:1007D800FF50010E8E098F0A780A740126F650041C
:1007E80018E436F6400302072A22054D22054C225A
:1007F800054EC2CF2290F800E4936406600280FEA2
:1008080075840175A70075FF80900788E4F075C9A5
:100818001075A70F75A1C775A70075D90075CEFF0C
:1008280075A70F75F1FE75F2FF75F33775F47875D6
:10083800A4BA75A5FF75A60775AE0075AFFF75D488
:100848008175D5FF75D6FF75D7FFC296C295C2A030
:10085800C297E5B554BFF5B5E5B554DFF5B5E5B5CF
:1008680054EFF5B5E5B5547FF5B5E5B554F7F5B5ED
:10087800E5B554FDF5B575A70075A20175A14775D5
:10088800F80975BC0175BE0475BD6C75BE0775BDEC
:10089800A075BE0875BD0175BC0075BB1875BC2078
:1008A80075BA0875E88075D11375A70F75E10575D8
:1008B800E20075C740759700759780740A1240EB7F
:1008C8007597C0E5975420700280F8758F0275A758
:1008D80000D2AF75980075A90C75A70F75AB437555
:1008E800ADFB75AC1E75A700758911758E00758CEA
:1008F80000758A00D2A9D28C758D00758B00D2AB99
:10090800D28E75CD0075CC0075CA0075CB00D2ADFE
:10091800C2CFD2CA7591047592007593CD75EF0652
:1009280075D94075CF01900786E4F0A3F0751300E0
:10093800751400C299D20AC20D12048174C8F51840
:100948007517001226E875A70FE5FB90001AF0E569
:10095800FA90001BF0E5F990001CF075A70090F8DC
:1009680000E493F50812281F122D59900789E0908A
:100978000026F090078AE0900027F090078BE0901F
:100988000028F090078CE0900029F090078DE0F5A2
:100998006690078EE0F56890078FE0F569900790FC
:1009A800E0F56A900791E0F565900792E0F56790A9
:1009B8000793E0F564900794E0F563900795E0905D
:1009C800002AF0900796E090002BF0900797E090AF
:1009D800002CF0900798E0900041F0900799E09083
:1009E8000042F090079AE0900043F090079BE09057
:1009F8000044F090079CE0900045F090079DE0903F
:100A08000046F090079EE0900047F090079FE09026
:100A18000048F09007A0E0900033F09007A1E09024
:100A28000034F09007A2E0900035F09007A3E09022
:100A38000036F07400900082F090013AE0700C905B
:100A4800013BE0700690013CE060028004C20A802D
:100A580002D20A90F807E493900021F0900021E078
:100A6800440A900021F0900021E054FE900021F00B
:100A78007406900012F07402900013F090F802E4EB
:100A880093900014F07403900015F074039000160E
:100A9800F07412900017F07405900018F09000148C
:100AA800E0B404067404900018F0900014E0B40355
:100AB800067403900018F07405900019F090F8047B
:100AC800E49390001DF0740090001EF090F805E487
:100AD8009390001FF090F806E493900020F074FFC4
:100AE800900022F0744A900125F07461900126F07C
:100AF8007474900127F07463900128F0746F90016A
:100B080029F0742090012AF0745290012BF074455A
:100B180090012CF0743490012DF0742090012EF087
:100B2800742090012FF07434900130F074539001C8
:100B380031F07450900132F07444900133F0900019
:100B48007AE0D394014006740090007AF075580159
:100B5800755901740390004CF01200C91204CA9030
:100B68000014E0B404051206568011900014E0D376
:100B7800940440051205888003120724122714E5FF
:100B8800B554FEF5B5900025E4F0900786E4F0A38F
:100B9800F0752400752300754800752A0075290032
:100BA800754900753200753100754A007554007535
:100BB8005500755A0075510475520175343C7533EA
:100BC80000757000756F007571CD7556007557000A
:100BD800754300754400754500754600755B0075E2
:100BE8004700754200754100900006E4F0A3F090BC
:100BF8000008E4F0A3F0755E00755F0090000E74C5
:100C0800FDF0A374E8F0900023E4F07464900024ED
:100C1800F0C200D201C202D203754D00756D00C248
:100C280094C293C287C290C291C20C7E017F009089
:100C38000028E0124119900027E02FFF50010E9084
:100C4800000AEEF0A3EFF0900026E0700674FF9023
:100C58000026F090000AE0FEA3E0FFEFD394FFEE39
:100C6800940F400790000AE4F0A3F074009000711C
:100C7800F07400900079F07400900082F074009095
:100C8800008DF074009000B4F0E567700375670498
:100C9800743A90074EF074FD90074FF09003D4E03B
:100CA800900414F0D2B0D2B7D2A7D2A6D2B1D2A3B0
:100CB800C207A2B6B39204A2B3B39205D29CD2ECF7
:100CC80075CF01A298B34005C2981230BDE51360F4
:100CD80006A299B3B340028005C29912362DE514D5
:100CE80064016005E514B4040280D5E54DD394058C
:100CF800400CE55AC394C85002055A754D00E57179
:100D0800C394F0501A786F12003FAE6FAF70EFD3F4
:100D180094E8EE940340080571757000756F00C281
:100D28008E7E047F00E54C124119E58D75F004A410
:100D3800FDACF0EF2DFDEE3CFCE58B75F04084FF3B
:100D48007E00ED2FFFEC3EFE8E258F26D28EA2B6BA
:100D5800300401B35003020E9BA2B6300401B35015
:100D680003020E9BA2B640670554A20D400575FF0D
:100D7800A0D20DE5B54401F5B5900024E4F0E554A2
:100D8800D3956640487C837DC2AE25AF26123FB915
:100D98008E238F24E5482FFF50010E740112410B5A
:100DA8008E238F24852448755401C28E758D007555
:100DB8008B00754C00D28E7403BE00039F500690C2
:100DC80000257401F0E543B40603754300D204A27C
:100DD800B6B35003020E9BC20490006BE060181279
:100DE800376EA200B34008E5B54408F5B58006E5BE
:100DF800B554F7F5B58002C20090006EE060181295
:100E080038C3A202B34008E5B54402F5B58006E54B
:100E1800B554FDF5B58006E5B554FDF5B5A207B3A3
:100E28004004D2878002C287900059E06004D290C3
:100E38008002C29090004AE0B40104D2948002C2B9
:100E480094900049E0B40104D2938002C293A209AD
:100E5800B34004D2918002C291900018E0FE900045
:100E680014E0C39E4009900014E0D394084009742C
:100E7800FB900023F012048190001DE060159000A3
:100E88001DE0FE900017E06E600974FE900023F0EC
:100E9800120481C2CA7E017F00E54E124119E5CDD8
:100EA8002FFF50010E8E278F28D2CAE565B401485E
:100EB80090000EE0FCA3E0FDEFC39DEE9C4039B22C
:100EC80008E52A45296013A208B34008E5B544049B
:100ED800F5B58006E5B554FBF5B590000EE0FEA328
:100EE800E0FF900010E0FCA3E0FDEF2DFDEE3CFCE0
:100EF80090000EECF0A3EDF0A2B3300501B350035F
:100F0800020FE9A2B3300501B35003020FE9A2B3FF
:100F18005003020FE20555A20D400575FFA0D20D42
:100F2800E5B54401F5B5900024E4F0E555D395689E
:100F38005003020FE07CEA7D60AE27AF28123FB96C
:100F48008E298F2AE56912411974FF8E048F05FFD7
:100F58001240FB8C298D2AE5492DFD50010C7401A6
:100F68008C068D0712410B8E298F2A852A49A209E2
:100F7800B340157464124119900067E08E048F0520
:100F8800FF1240FB8C298D2A75550190000EE0FE5A
:100F9800A3E0FFAC27AD2812000390000EEEF0A3EB
:100FA800EFF0E567FF1240FB740AFF1240FB900068
:100FB8007BE08C068D0712411974148E048F05FF8F
:100FC8001240FB900010ECF0A3EDF0C2CA75CD0002
:100FD80075CC00754E00D2CAD205A2B3B34002C286
:100FE80005900025E0B40107E556C39406400302C6
:100FF80015FDE56D9026ACF8282873900059E0C3DC
:1010080094024003021157E551D394015003021191
:1010180057E55175F040A4FFAEF090031212001E80
:10102800E0C395455018E55175F040A4FFAEF09027
:10103800031112001EE0F52E752D00021157E5511F
:1010480075F040A4FFAEF090031012001EE0C395A7
:101058004540030210F3E55175F040A4FFAEF0904F
:10106800031112001EE55175F040A4FFAEF0E0FC3C
:1010780090030F12001EECFEE0FFEEC39FFEE55149
:101088008E0475F040A4FFAEF090031012001EE02D
:10109800F40425458C0088F0A4FFAEF0E5518F04D8
:1010A8008E0575F040A4FFAEF090031212001EE505
:1010B8005175F040A4FFAEF0E0FA90031012001E44
:1010C800EAFEE0FFEEC39FFECDCCCD8E071240FBBB
:1010D800E55175F040A4FFAEF090030F12001EE03A
:1010E8002DFD50010C8C2D8D2E8064E55175F0403E
:1010F800A4FFAEF090030F12001EE55175F040A456
:10110800FFAEF0E0FC90030E12001EECFEE0FFEED6
:10111800C39F8545F0A4FFAEF0E5518F048E057599
:10112800F040A4FFAEF090031012001EE0FECDCCFC
:10113800CD8E071240FBE55175F040A4FFAEF0904C
:10114800030E12001EE02DFD50010C8C2D8D2E7506
:101158006D010215FD900059E0C39402400302138B
:101168000B90004FE0D3955150030212B3E551752F
:10117800F040A4FFAEF090031812001EE0C395459E
:101188005018E55175F040A4FFAEF0900317120017
:101198001EE0F52C752B000212B3E55175F040A442
:1011A800FFAEF090031612001EE0C39545400302FF
:1011B800124FE55175F040A4FFAEF09003171200EE
:1011C8001EE55175F040A4FFAEF0E0FC9003151247
:1011D800001EECFEE0FFEEC39FFEE5518E0475F0A5
:1011E80040A4FFAEF090031612001EE0F40425455B
:1011F8008C0088F0A4FFAEF0E5518F048E0575F0E1
:1012080040A4FFAEF090031812001EE55175F0409F
:10121800A4FFAEF0E0FA90031612001EEAFEE0FF0B
:10122800EEC39FFECDCCCD8E071240FBE55175F085
:1012380040A4FFAEF090031512001EE02DFD5001F2
:101248000C8C2B8D2C8064E55175F040A4FFAEF01A
:1012580090031512001EE55175F040A4FFAEF0E0B2
:10126800FC90031412001EECFEE0FFEEC39F8545C0
:10127800F0A4FFAEF0E5518F048E0575F040A4FF91
:10128800AEF090031612001EE0FECDCCCD8E0712F4
:1012980040FBE55175F040A4FFAEF0900314120036
:1012A8001EE02DFD50010C8C2B8D2CE551B4012333
:1012B800E560D39401401CE55604D395514014E5EC
:1012C80045C39405500D90035FE0A829B800069522
:1012D8002A40028003755102E551B5602290004F03
:1012E800E0D395514019E55175F040A4FFAEF09058
:1012F800031712001EE0A823B800069524400280B8
:10130800020560756D020215FD900059E0B4022ACD
:10131800E55175F040A4FFAEF090031712001EE0EF
:10132800F52C752B00E55175F040A4FFAEF0900345
:101338000E12001EE0F52E752D00900059E0B40342
:101348000F900051E0F52C752B00752E00752D00BF
:10135800756D030215FDE55175F040A4FFAEF090E0
:10136800032012001EE0C3955A4003021433900074
:1013780049E07036E551D394014029AE23AF24AC3F
:101388002DAD2EEDD39FEC9E401AE55175F040A48B
:10139800FFAEF090031E12001EE0A829B80005D386
:1013A800952A5002800215518034E551D3940240A9
:1013B80029AE23AF24AC2DAD2EEDD39FEC9E401A61
:1013C800E55175F040A4FFAEF090031E12001EE038
:1013D800A829B80005D3952A500280021551E55175
:1013E800B55237E551C395605030E55604D3955151
:1013F8004028AE23AF24AC2BAD2CEFD39DEE9C4000
:1014080019E55175F040A4FFAEF090031F12001EBD
:10141800E0A829B80006952A400280020551C29228
:10142800E55165526005C207755A00756D040215CD
:10143800FDE55175F040A4FFAEF090031A12001EAE
:10144800E0B40117E55175F040A4FFAEF090032019
:1014580012001EE0240AC3955A400302150975308C
:1014680064752F00A207B3500B900060E02405C3F9
:1014780095454003021509E55175F040A4FFAEF00B
:1014880090031D12001EE0C395454064E55175F0B8
:1014980040A4FFAEF090031C12001EE55175F04009
:1014A800A4FFAEF0E0FC90031B12001EECFEE0FF70
:1014B800EEC39F8545F0A4FFAEF0E5518F048E057D
:1014C80075F040A4FFAEF090031D12001EE0FECDA3
:1014D800CCCD8E071240FBE55175F040A4FFAEF06D
:1014E80090031B12001EE02DFD50010C8C2F8D3037
:1014F800AE23AF24AC2FAD30EFD39DEE9C4002D28B
:1015080007756D050215FDE551B40109900059E014
:10151800C3940240030215DD900358E0D39545506B
:10152800030215DD900356E0C395455040900357DC
:10153800E0FE900355E0F4042EFE900356E0F40418
:1015480025458E0088F0A4FFAEF0900358E0FC908B
:101558000356E0F4042C8E048F05FF1240FB900321
:1015680055E02DFD50010C8C2B8D2C802C900355B3
:10157800E0FE900354E0F4042E8545F0A4FFAEF09D
:10158800900356E08E048F05FF1240FB900354E051
:101598002DFD50010C8C2B8D2CE551C395605030DE
:1015A800E55604D395514028AE23AF24AC2BAD2C7F
:1015B800EFD39DEE9C4019E55175F040A4FFAEF0C5
:1015C80090031F12001EE0A829B80006952A4002C1
:1015D8008003755102900049E0B40106E5516401A9
:1015E80060028003755102E55165526005C20775B6
:0515F8005A00756D00B2
:1026AC0002100302115D02131102135E02143902AF
:0226BC00150FF8
:1015FD00900050E02402A823B80007D395244002A0
:10160D00C207900025E0B40109900059E0C394038E
:10161D004003021785900049E060030216D4E5519E
:10162D00D394014034E55175F040A4FFAEF0900322
:10163D001412001EE0A823B8001FD39524401AE50C
:10164D005175F040A4FFAEF090031F12001EE0A8EC
:10165D0029B80005D3952A500280021551E551D3C2
:10166D009401402FE55175F040A4FFAEF0900312A8
:10167D0012001EE0C39545501AE55175F040A4FFC8
:10168D00AEF090031E12001EE0A829B80005D395F8
:10169D002A500280021551E551D394014022E5569E
:1016AD0004C39551501AE55175F040A4FFAEF0906A
:1016BD00031E12001EE0A829B80005D3952A50027A
:1016CD008002155102177AE551D394024034E55149
:1016DD0075F040A4FFAEF090031412001EE0A82395
:1016ED00B8001FD39524401AE55175F040A4FFAE04
:1016FD00F090031F12001EE0A829B80005D3952A0B
:10170D00500280021551E551D39402402FE55175D9
:10171D00F040A4FFAEF090031212001EE0C39545F9
:10172D00501AE55175F040A4FFAEF090031E120063
:10173D001EE0A829B80005D3952A50028002155144
:10174D00E551D394024022E55604C39551501AE554
:10175D005175F040A4FFAEF090031E12001EE0A8DC
:10176D0029B80005D3952A500280021551E551651F
:10177D00526005C207755A00900060E0D395455040
:10178D0009900054E0C395455002C207900059E0FE
:10179D0070030219EAA2A5B34008A2A4B340030244
:1017AD0019D3AE35AF367441D39F749C9E400578E6
:1017BD003512003FAE35AF36EFB48806EEB41302E6
:1017CD0080030219B0A2A55003021873900059E0CE
:1017DD00B4010B90004FE0D395604002056090007E
:1017ED0059E0B40254E55175F040A4FFAEF09003FA
:1017FD002012001EE0C3955A503F90004FE0D39544
:10180D00514021E55604D395514019E55175F040ED
:10181D00A4FFAEF090031412001EE0A823B800063A
:10182D00952440028002055190004FE0F560E5518E
:10183D0065526005C207755A00900059E0B4032641
:10184D0090004FE0D395514008E55604D395515083
:10185D00028002055190004FE0F560E55165526040
:10186D0005C207755A00A2A450030219B090005981
:10187D00E0B4016E900049E07035E551D39401401C
:10188D0029E55175F040A4FFAEF090031E12001E25
:10189D00E0A829B8000FD3952A400A1551755A00B2
:1018AD00855160800385516080037560018033E54B
:1018BD0051D394024029E55175F040A4FFAEF0904C
:1018CD00031E12001EE0A829B8000FD3952A400A66
:1018DD001551755A008551608003855160800375DF
:1018ED006002900059E0D3940150030219A4E55110
:1018FD0075F040A4FFAEF090032012001EE0C395DA
:10190D005A40030219A4900049E07041E551D39467
:10191D00014034E55175F040A4FFAEF09003111273
:10192D00001EE0A823B8001FD39524401AE5517579
:10193D00F040A4FFAEF090031E12001EE0A829B8DF
:10194D000005D3952A500280021551803FE551D3F1
:10195D0094024034E55175F040A4FFAEF0900311B0
:10196D0012001EE0A823B8001FD39524401AE5519C
:10197D0075F040A4FFAEF090031E12001EE0A829E2
:10198D00B80005D3952A500280021551E5516552D4
:10199D006005C207755A00E556B40704055E80035D
:1019AD00755E00E563B4010EAE35AF36EF64407081
:1019BD0005EE649C6002800EA2A54003755801A23D
:1019CD00A44003755802A2A5B3B35006A2A4B3B3A5
:1019DD0040028006753600753500021AD8A2A5B3EF
:1019ED004008A2A4B34003021AC4AE35AF36744109
:1019FD00D39F749C9E4005783512003FAE35AF36AF
:101A0D00EFB48806EEB413028003021AC4A2A540F7
:101A1D006F900068E0605A90004AE0B401079000B2
:101A2D004AE4F0800690004A7401F090004AE0709C
:101A3D0005756003800375600490004AE0B40104ED
:101A4D00D2948002C294E551B4041AE55175F04068
:101A5D00A4FFAEF090031E12001EE0A829B80005E9
:101A6D00D3952A50028008755103C207755A00801C
:101A7D0003756004E556B40704055E8003755E00CA
:101A8D00A2A44033900069E06021900049E0B401C8
:101A9D0007900049E4F080069000497401F0900031
:101AAD0049E0B40104D2938002C293E556B4070411
:101ABD00055E8003755E00A2A5B3B35006A2A4B364
:101ACD00B340028006753600753500E558655960DE
:101ADD0006900082E06003021C60C29C75140075C4
:101AED001300C2CAE5589026BEF82828738012123A
:101AFD002D59800D122E328008122F0B8003122FBC
:011B0D00E4F3
:0F26BE00021AFA021AFC021B01021B06021B0B76
:101B0E00900029E090007AF0E566900057F0E568C5
:101B1E00900062F0E569900063F0E56A900074F061
:101B2E00E56590007CF0E56790007DF0E56490003F
:101B3E0080F0E563900081F090002AE090013AF089
:101B4E0090002BE090013BF090002CE090013CF0D7
:101B5E00900041E0900090F0900042E0900091F0F3
:101B6E00900043E0900092F0900044E0900093F0DB
:101B7E00900045E0900094F0900046E0900095F0C3
:101B8E00900047E0900096F0900048E0900097F0AB
:101B9E00900033E0900099F0900034E090009AF0BD
:101BAE00900035E090009BF0900036E090009CF0A5
:101BBE007400900082F0744A900125F074619001D7
:101BCE0026F07474900127F07463900128F0746FFE
:101BDE00900129F0742090012AF0745290012BF09C
:101BEE00744590012CF0743490012DF07420900106
:101BFE002EF0742090012FF07434900130F0745355
:101C0E00900131F07450900132F07444900133F031
:101C1E009003D4E0900414F0743A90074EF074FDE3
:101C2E0090074FF01200C9900004E4F0A3F090006A
:101C3E00067475F0A37430F09000087475F0A374F8
:101C4E0030F0855859D2CA754C00D29C741B900046
:101C5E0023F0E556C394065005E551B55202804E69
:101C6E00C207E55175F040A4FFAEF09003221200BA
:101C7E001EE030E003D38001C39296E55175F0402B
:101C8E00A4FFAEF090032312001EE030E003D380D9
:101C9E0001C39295855152AE29AF2A7405BE000339
:101CAE009F5007E545D3940550028002D292E55627
:101CBE00D394055003021D85C207E551D39401400C
:101CCE0059E55175F040A4FFAEF090031E12001EB0
:101CDE00E0A829B80007D3952A40021551E55165B1
:101CEE00526035E55175F040A4FFAEF0900322121C
:101CFE00001EE030E003D38001C39296E55175F0EB
:101D0E0040A4FFAEF090032312001EE030E003D398
:101D1E008001C39295855152805DE556B4061A90A6
:101D2E0000ACE030E003D38001C392969000ADE0AA
:101D3E0030E003D38001C39295E556B4071A9000A4
:101D4E00A5E030E003D38001C392969000A6E03068
:101D5E00E003D38001C39295E556B4081A90009E15
:101D6E00E030E003D38001C3929690009FE030E014
:101D7E0003D38001C39295900072E06058E54575DB
:101D8E00F00284FF7E0090014E12001EE0F55CE52D
:101D9E004775F00A84FF7E0090024E12001EE0F599
:101DAE005DE55C255DD39464400BE55C255DC394D5
:101DBE0064F55C8003755C00E55C75F00284FF7E63
:101DCE00008F5CEFC394335007EF24CDF55C800396
:101DDE00755CFF801CE54575F00284FF7E00900166
:101DEE004E12001EE075F00284FF7E00EF24CDF54A
:101DFE005CE595C3955C4004C2A28002D2A2A20704
:101E0E00B34005E556B407037571CDE595C39571DD
:101E1E004004C2A18002D2A1E543C394064003024E
:101E2E002484A2EDB35003022484C2EDE543600383
:101E3E00021F8B7E017F00E5BE124119E5BD2FFF0B
:101E4E0050010E900000EEF0A3EFF0900029E0B4E8
:101E5E0001177E0F7FFF900000E0FCA3E0FD120053
:101E6E0003900000EEF0A3EFF0900079E0B4025B77
:101E7E00900000E0FEA3E0FF90000AE0FCA3E0FD6E
:101E8E00EDD39FEC9E400F900000E0F8A3E0900091
:101E9E000AC8F0A3C8F0900000E0FEA3E0FF900097
:101EAE000CE0FCA3E0FDEFD39DEE9C400F900000F4
:101EBE00E0F8A3E090000CC8F0A3C8F0900000E09A
:101ECE00FEA3E0FF740412410B8F44900079E07082
:101EDE0060900000E0FEA3E0FF90000AE0FCA3E0AB
:101EEE00FDEFD39DEE9C400D120003900000EEF02E
:101EFE00A3EFF08007900000E4F0A3F0900000E064
:101F0E00FEA3E0FF7410124119900026E08E048F9C
:101F1E0005FF1240FB900000ECF0A3EDF07400D32F
:101F2E009D74019C4008900001E0F54480037544C7
:101F3E00FFE54475F00AA4FFAEF074198E048F0508
:101F4E00FF1240FB8D45ED2532FFAE3150010E7470
:101F5E000112410B8F45854532753100EFD39462E6
:101F6E004003754562900072E06401600690006661
:101F7E00E060028005754301800375BB17E543B42D
:101F8E000102800302207B7E017F00E5BE12411913
:101F9E00E5BD2FFF50010E900000EEF0A3EFF09084
:101FAE000072E0B4017EE53445336025AC33AD34C8
:101FBE001DBDFF011C8F028E038C068D07903DB94F
:101FCE0012002EE493FE740193FFEFC39AEE9B4032
:101FDE000280057833124143AE33AF3474B3BE0082
:101FEE0025D39F4021900000E0FCA3E0FD0FBF0031
:101FFE00010E903DB912002EE493FE740193FFED95
:10200E00C39FEC9E40028005783312003FAE33AF83
:10201E0034E56A12411974648E048F05FF1240FB79
:10202E008D478033900066E0602D900000E0FEA3A7
:10203E00E0FFEFD39400EE9408400F900066E0B4FA
:10204E000104C2098002D209800D900066E0B4013D
:10205E0004D2098002C209900072E0640260069008
:10206E000066E0600575BB168003754302E543B458
:10207E00020280030221697E017F00E5BE12411932
:10208E00E5BD2FFF50010E900000EEF0A3EFF09093
:10209E000072E0B4027EE53445336025AC33AD34D6
:1020AE001DBDFF011C8F028E038C068D07903C4FC9
:1020BE0012002EE493FE740193FFEFC39AEE9B4041
:1020CE000280057833124143AE33AF3474B3BE0091
:1020DE0025D39F4021900000E0FCA3E0FD0FBF0040
:1020EE00010E903C4F12002EE493FE740193FFED0F
:1020FE00C39FEC9E40028005783312003FAE33AF93
:10210E0034E56A12411974648E048F05FF1240FB88
:10211E008D478033900066E0602D900000E0FEA3B6
:10212E00E0FFEFD39400EE9408400F900066E0B409
:10213E000104C2098002D209800D900066E0B4014C
:10214E0004D2098002C209900072E0700375470044
:10215E00900066E07002C20975BB1FE543B40345EB
:10216E007E017F00E5BE124119E5BD2FFF50010E25
:10217E00900000EEF0A3EFF0740912411974E68E90
:10218E00048F05FF1240FB8C418D42E54A2DFD5018
:10219E00010C74018C068D0712410B8E418F428506
:1021AE00424A75BB19E543B40402800302236C7ED8
:1021BE00017F00E5BE124119E5BD2FFF50010E90C3
:1021CE000000EEF0A3EFF0740412410B8F4BE564A8
:1021DE00B40102800302229E756B00756B00E56BE5
:1021EE00D39407400302228BE56B900041124131DC
:1021FE00E0D3954B501AE56B900041124131E0F45B
:10220E0004254BFEE56B900037124131EEF080173E
:10221E00E56B900041124131E0C3954BFEE56B90AA
:10222E000037124131EEF0E56BC394044009900083
:10223E0084E0C3956B503BE56B6029E56B900037EE
:10224E00124131FEE0FFEE90003FE0D39F4013E5D8
:10225E006B900037124131E090003FF0E56B90003B
:10226E0040F0800E900037E090003FF07400900038
:10227E0040F0786B740126F640030221EC9000408A
:10228E00E0F4042408F556E556D394054002C292B4
:10229E00E564D39401402FE54BD3946E4004D20EE7
:1022AE008002C20E755605E564B40205A20EB34057
:1022BE00028003755607E564B40306A20EB3B3405D
:1022CE00028003755607E55765566008E55104F51B
:1022DE0052855657E5569026CDF82828738050D251
:1022EE00A0804CE544C394585004D2A08002C2A0F2
:1022FE00803DE551C394045007E544C39458400211
:10230E008004D2A08002C2A080258023E551C39410
:10231E00045007E544C3945840028004D2A08002C2
:0F232E00C2A0E551B40402D2A080048002800056
:1026CD000222EB0222ED0222F10223000223180264
:0B26DD00231A02233902233B02233D95
:10233D00E556B40708E5B54480F5B58006E5B55416
:10234D007FF5B5E55664066005E556B40808E5B5B4
:10235D004410F5B58006E5B554EFF5B575BB13E53D
:10236D0043B4050280030224807E017F00E5BE1286
:10237D004119E5BD2FFF50010E900000EEF0A3EFC7
:10238D00F0740412410B8F46E563B4020280030220
:10239D00247D756B00756B00E56BD39403400302D0
:1023AD002434E56B900033124131E0D39546501A39
:1023BD00E56B900033124131E0F4042546FEE56BE8
:1023CD0090002D124131EEF08017E56B9000331225
:1023DD004131E0C39546FEE56B90002D124131EE83
:1023ED00F0E56B6029E56B90002D124131FEE0FFA9
:1023FD00EE900031E0D39F4013E56B90002D12411C
:10240D0031E0900031F0E56B900032F0800E9000DD
:10241D002DE0900031F07400900032F0786B740173
:10242D0026F640030223A5900082E07043E52A457D
:10243D00296036E558C39403500A900032E004C376
:10244D00940340028007900032E004F558E558D31C
:10245D009402400A900032E004D3940250028007A7
:10246D00900032E004F5588007900032E004F558F2
:10247D0075BB180543D2ECE55ED3940450030225D9
:10248D006C75CF01C2A2AE35AF367488D39F74136D
:10249D009E4005A2A5B34014AE35AF367488D39FC8
:1024AD0074139E4005A2A4B34002804878351200F3
:1024BD003FAE35AF36EFB4883BEEB41337A2A5B3BC
:1024CD00500990004FE0D395515002800405518082
:1024DD0011A2A5B3500890004FE065516002800233
:1024ED00D207A2A4B35007E551D394015002800442
:1024FD001551C207A2A5B3B35006A2A4B3B34002AF
:10250D008006753600753500E55165526035E5512B
:10251D0075F040A4FFAEF090032212001EE030E0F3
:10252D0003D38001C39296E55175F040A4FFAEF040
:10253D0090032312001EE030E003D38001C3929577
:10254D00855152A20740057571CD80037571FFE568
:10255D0095C395714004C2A18002D2A102248EA21E
:10256D000DB3500DAE25AF2674E8C39F74039E4086
:10257D0002800575FFA0D20DAE25AF26EFD39420B6
:10258D00EE944E5003022680120481C28E758D008A
:10259D00758B00754C00D28EC207757000756F007B
:1025AD007571CD7551047524007523007554007532
:1025BD005A00C287900059E06004D2908002C29008
:1025CD0090004AE0B40104D2948002C29490004974
:1025DD00E0B40104D2938002C293A209B34004D2A5
:1025ED00918002C29190006BE0601812376EA200CC
:1025FD00B34008E5B54408F5B58006E5B554F7F5E3
:10260D00B58002C20090006EE060181238C3A202BD
:10261D00B34008E5B54402F5B58006E5B554FDF5C2
:10262D00B58006E5B554FDF5B590000E74FDF0A32B
:10263D0074E8F0E543B40603754300900025E4F01B
:10264D00752600752500758D00758B00754C0090F5
:10265D000024E0C394035008900024E004F08006A9
:10266D007403900024F0900024E0B40306E5B55403
:10267D00FEF5B5AE27AF28EFD39410EE9427401C8E
:10268D00C2CA75CD0075CC00752800752700D2CA59
:0F269D00754E00752A00752900755500020CC88E
:103A75000000010001320164019601960200021264
:103A850002240200020003000340038003C0040077
:103A95000440048004C00500060006000600060078
:103AA500060006000600060000FF013101630195CE
:103AB50001FF01FF0211022302FF02FF02FF033F84
:103AC500037F03BF03FF043F047F04BF04FF05FF1B
:103AD50006FF06FF06FF06FF06FF06FF06FF06FFB9
:103AE5000FAA0FA50F9F0F9A0F940F8D0F870F80A9
:103AF5000F780F710F680F600F570F4E0F450F3B73
:103B05000F300F250F1A0F0E0F020EF50EE80EDB04
:103B15000ECC0EBE0EAE0E9F0E8E0E7D0E6C0E5A88
:103B25000E470E340E200E0C0DF70DE20DCB0DB524
:103B35000D9D0D850D6D0D540D3A0D200D050CE9EE
:103B45000CCE0CB10C940C760C580C3A0C1B0BFBE0
:103B55000BDB0BBB0B9A0B790B570B350B130AF1D0
:103B65000ACE0AAB0A870A640A400A1C09F809D476
:103B750009B0098C09670943091F08FB08D608B273
:103B8500088E086A0846082307FF07DC07B9079669
:103B950007730751072F070D06EC06CA06AA068903
:103BA50006690649062A060A05EC05CD05B0059203
:103BB50005750558053C0520050504EA04CF04B53F
:103BC500049C04820469045104390422040B03F49F
:103BD50003DE03C803B2039D038903750361034D27
:103BE500033B03280316030402F202E102D102C0DB
:103BF50002B002A0029102820273026502570249D5
:103C0500023C022F02220216020901FD01F201E621
:103C150001DB01D001C601BB01B101A7019D0194E2
:103C2500018B018201790170016801600158015021
:103C35000148014101390132012B0125011E0118FD
:103C45000111010B010500FF00FA0FA60FA00F9946
:103C55000F920F8B0F840F7C0F740F6B0F620F5831
:103C65000F4E0F430F380F2C0F1F0F120F050EF7B6
:103C75000EE80ED80EC80EB70EA50E930E800E6C6C
:103C85000E580E420E2C0E150DFD0DE40DCB0DB18B
:103C95000D950D790D5D0D3F0D200D010CE10CC04D
:103CA5000C9E0C7C0C590C350C100BEA0BC40B9EAE
:103CB5000B760B4F0B260AFD0AD40AAA0A800A5571
:103CC5000A2A09FF09D409A8097C0950092508F918
:103CD50008CD08A10875084A081E07F307C8079DFF
:103CE50007730749072006F706CE06A6067E065780
:103CF5000630060A05E405BF059B05770554053220
:103D0500051004EF04CE04AE048F0471045304358A
:103D1500041903FD03E203C703AD0394037B0363A7
:103D2500034B0334031E030802F302DE02CA02B684
:103D350002A30291027F026D025C024C023C022C3E
:103D4500021D020E020001F201E401D701CA01BE03
:103D550001B101A6019A018F0185017A0170016601
:103D6500015D0153014A0141013901310129012157
:103D750001190112010B010400FD00F700F000EA32
:103D850000E400DE00D900D300CE00C900C400BFA6
:103D950000BA00B500B100AD00A800A400A0009CC9
:103DA500009900950091008E008A008700840081AB
:043DB500007E007B11
:1026E800751A00751900AE19AF1AAC17AD18EDC3FD
:1026F8009FEC9E401674FF1240EB75CF01781A7458
:102708000126F6500418E436F650DB22900786E4DA
:10271800F0A3F0751000750F00751300751400C252
:102728000FD21022C2AF75D900758F0375B7A57582
:10273800B7F190F800E4F0758F0175B7A575B7F19A
:10274800E50890F800F075B7A575B7F190F801E4C1
:10275800F075B7A575B7F190079DE090F802F07590
:10276800B7A575B7F19007A1E090F803F075B7A584
:1027780075B7F190079EE090F804F075B7A575B7A6
:10278800F190079FE090F805F075B7A575B7F1903F
:1027980007A0E090F806F075B7A575B7F19007A205
:1027A800E090F807F0758F0075D940D2AF229007F6
:1027B80088E0B4AB61C2AF75D90075B62275F52251
:1027C800758F0375B7A575B7F1740090F600F075AD
:1027D8008F01750A00750900AE09AF0A7413BE00AF
:1027E800279F402475B7A575B7F190078912001E79
:1027F800E0FC90F60012001EECF0780A740126F650
:10280800500418E436F650D0758F0075F51175B67A
:102818002075D940D2AF22C2AF75D90075F522759F
:102828000A00750900AE09AF0A7413BE00229F4062
:102838001F90F60012001EE493FC90078912001EF8
:10284800ECF0780A740126F6500418E436F650D5F0
:1028580075F51175D940D2AF22900788E0B4AA0265
:10286800800302299EC2AF75D90075B62275F5227C
:10287800758F0375B7A575B7F1740090EE00F07504
:10288800B7A575B7F1740090F000F075B7A575B7E6
:10289800F1740090F200F075B7A575B7F174009067
:1028A800F400F0758F01750A00750900AE09AF0ACA
:1028B80074FFC39F74019E402475B7A575B7F19046
:1028C800004E12001EE0FC90EE0012001EECF078A4
:1028D8000A740126F6500418E436F650CF750A003B
:1028E800750900AE09AF0A74FFC39F74019E4024A6
:1028F80075B7A575B7F190024E12001EE0FC90F076
:102908000012001EECF0780A740126F6500418E450
:1029180036F650CF750A00750900AE09AF0A74FF84
:10292800C39F74019E402475B7A575B7F190044EF6
:1029380012001EE0FC90F20012001EECF0780A74FF
:102948000126F6500418E436F650CF750A007509CA
:1029580000AE09AF0A74FFC39F74019E402475B787
:10296800A575B7F190064E12001EE0FC90F4001217
:10297800001EECF0780A740126F6500418E436F6C6
:1029880050CF758F0075F51175B62075D940D2AF47
:10299800743A90074EF022900788E0B4AA028003A8
:1029A800022ADCC2AF75D90075B62275F522758F7B
:1029B8000375B7A575B7F1740090E600F075B7A573
:1029C80075B7F1740090E800F075B7A575B7F174A4
:1029D8000090EA00F075B7A575B7F1740090EC00A7
:1029E800F0758F01750A00750900AE09AF0A74FF0A
:1029F800C39F74019E402475B7A575B7F190004E2A
:102A080012001EE0FC90E60012001EECF0780A743A
:102A18000126F6500418E436F650CF750A007509F9
:102A280000AE09AF0A74FFC39F74019E402475B7B6
:102A3800A575B7F190024E12001EE0FC90E8001256
:102A4800001EECF0780A740126F6500418E436F6F5
:102A580050CF750A00750900AE09AF0A74FFC39F0D
:102A680074019E402475B7A575B7F190044E120005
:102A78001EE0FC90EA0012001EECF0780A740126B1
:102A8800F6500418E436F650CF750A00750900AE02
:102A980009AF0A74FFC39F74019E402475B7A575DA
:102AA800B7F190064E12001EE0FC90EC0012001EDA
:102AB800ECF0780A740126F6500418E436F650CF84
:102AC800758F0075F51175B62075D940D2AF743A77
:102AD80090074EF022900788E0B4AA028003022CE7
:102AE8001AC2AF75D90075B62275F522758F0375B0
:102AF800B7A575B7F1740090DE00F075B7A575B786
:102B0800F1740090E000F075B7A575B7F174009006
:102B1800E200F075B7A575B7F1740090E400F075A0
:102B28008F01750A00750900AE09AF0A74FFC39FCB
:102B380074019E402475B7A575B7F190004E120038
:102B48001EE0FC90DE0012001EECF0780A740126EC
:102B5800F6500418E436F650CF750A00750900AE31
:102B680009AF0A74FFC39F74019E402475B7A57509
:102B7800B7F190024E12001EE0FC90E00012001E19
:102B8800ECF0780A740126F6500418E436F650CFB3
:102B9800750A00750900AE09AF0A74FFC39F740176
:102BA8009E402475B7A575B7F190044E12001EE03B
:102BB800FC90E20012001EECF0780A740126F65030
:102BC8000418E436F650CF750A00750900AE09AF4F
:102BD8000A74FFC39F74019E402475B7A575B7F1A9
:102BE80090064E12001EE0FC90E40012001EECF06D
:102BF800780A740126F6500418E436F650CF758F1B
:102C08000075F51175B62075D940D2AF743A9007A2
:102C18004EF022900788E0B4AA028003022D58C221
:102C2800AF75D90075B62275F522758F0375B7A5EE
:102C380075B7F1740090D600F075B7A575B7F17443
:102C48000090D800F075B7A575B7F1740090DA0058
:102C5800F075B7A575B7F1740090DC00F0758F01B9
:102C6800750A00750900AE09AF0A74FFC39F7401A5
:102C78009E402475B7A575B7F190004E12001EE06E
:102C8800FC90D60012001EECF0780A740126F6506B
:102C98000418E436F650CF750A00750900AE09AF7E
:102CA8000A74FFC39F74019E402475B7A575B7F1D8
:102CB80090024E12001EE0FC90D80012001EECF0AC
:102CC800780A740126F6500418E436F650CF750ACF
:102CD80000750900AE09AF0A74FFC39F74019E40D6
:102CE8002475B7A575B7F190044E12001EE0FC904C
:102CF800DA0012001EECF0780A740126F650041867
:102D0800E436F650CF750A00750900AE09AF0A74AB
:102D1800FFC39F74019E402475B7A575B7F190064F
:102D28004E12001EE0FC90DC0012001EECF0780A47
:102D3800740126F6500418E436F650CF758F0075E6
:102D4800F51175B62075D940D2AF743A90074EF098
:102D580022C2AF75D90075F522750A00750900AE53
:102D680009AF0A74FFC39F74019E401F90EE0012C2
:102D7800001EE493FC90004E12001EECF0780A74DA
:102D88000126F6500418E436F650D4750A00750981
:102D980000AE09AF0A74FFC39F74019E401F90F0F4
:102DA8000012001EE493FC90024E12001EECF07814
:102DB8000A740126F6500418E436F650D4750A0051
:102DC800750900AE09AF0A74FFC39F74019E401FC6
:102DD80090F20012001EE493FC90044E12001EECC8
:102DE800F0780A740126F6500418E436F650D475C3
:102DF8000A00750900AE09AF0A74FFC39F74019EEB
:102E0800401F90F40012001EE493FC90064E12003E
:102E18001EECF0780A740126F6500418E436F650D1
:102E2800D475F51175D940D2AF22C2AF75D90075E6
:102E3800F522750A00750900AE09AF0A74FFC39F31
:102E480074019E401F90E60012001EE493FC90005F
:102E58004E12001EECF0780A740126F6500418E4AD
:102E680036F650D4750A00750900AE09AF0A74FF2A
:102E7800C39F74019E401F90E80012001EE493FC5B
:102E880090024E12001EECF0780A740126F65004E7
:102E980018E436F650D4750A00750900AE09AF0A71
:102EA80074FFC39F74019E401F90EA0012001EE445
:102EB80093FC90044E12001EECF0780A740126F67A
:102EC800500418E436F650D4750A00750900AE09A6
:102ED800AF0A74FFC39F74019E401F90EC0012005C
:102EE8001EE493FC90064E12001EECF0780A740162
:102EF80026F6500418E436F650D475F51175D94005
:102F0800D2AF22C2AF75D90075F522750A007509CE
:102F180000AE09AF0A74FFC39F74019E401F90DE84
:102F28000012001EE493FC90004E12001EECF07894
:102F38000A740126F6500418E436F650D4750A00CF
:102F4800750900AE09AF0A74FFC39F74019E401F44
:102F580090E00012001EE493FC90024E12001EEC5A
:102F6800F0780A740126F6500418E436F650D47541
:102F78000A00750900AE09AF0A74FFC39F74019E69
:102F8800401F90E20012001EE493FC90044E1200D1
:102F98001EECF0780A740126F6500418E436F65050
:102FA800D4750A00750900AE09AF0A74FFC39F748F
:102FB800019E401F90E40012001EE493FC90064E10
:102FC80012001EECF0780A740126F6500418E43654
:102FD800F650D475F51175D940D2AF22C2AF75D964
:102FE8000075F522750A00750900AE09AF0A74FF6D
:102FF800C39F74019E401F90D60012001EE493FCEC
:1030080090004E12001EECF0780A740126F6500467
:1030180018E436F650D4750A00750900AE09AF0AEF
:1030280074FFC39F74019E401F90D80012001EE4D5
:1030380093FC90024E12001EECF0780A740126F6FA
:10304800500418E436F650D4750A00750900AE0924
:10305800AF0A74FFC39F74019E401F90DA001200EC
:103068001EE493FC90044E12001EECF0780A7401E2
:1030780026F6500418E436F650D4750A007509008F
:10308800AE09AF0A74FFC39F74019E401F90DC0015
:1030980012001EE493FC90064E12001EECF0780A13
:1030A800740126F6500418E436F650D475F51175F7
:1030B800D940D2AF22E51464046006E59964FF6044
:1030C800028031A20F4004D20F8027E514600874F3
:1030D800E62514900023F0E513600874F02513909A
:1030E8000023F0E514B4010280FE75140075130086
:1030F800C20F8002C20FE514903A18F82828737599
:103108001400E599B4FF03751301E599B4FE03753E
:103118001302E599B4FD03751303E599B4FC03752F
:103128001304E599B4FA03751305E599B4FB06751C
:103138001401120481E599B4F90675140412048186
:10314800E599D394E54007E599C394F040028016C9
:103158008599157514027E017F00E515C394E61262
:1031680041198E0D8F0E900786E4F0A3F0E599D3F0
:1031780094C44007E599C394E640028028859915D0
:1031880075140374E5C39515F50E750D00AE0DAFF6
:103198000E903A7512002EE493F874019390078606
:1031A800C8F0A3C8F0D29902362C900786E0FEA397
:1031B800E0FFEFC39400EE94054009EFD394FFEECF
:1031C80094064013900786E0FEA3E0FF90004E129D
:1031D800001EE599F0800385996C90078612000E11
:1031E800900786E0FEA3E0FFEFB40106EEB4070205
:1031F800800302343C90074EE0B43C028003023462
:103208003CA20AB35005A20BB3400302332FC29C61
:1032180090007AE090078CF0900057E090078DF0CE
:10322800900062E090078EF0900063E090078FF0C6
:10323800900074E0900790F090007CE0900791F087
:1032480090007DE0900792F0900080E0900793F066
:10325800900081E0900794F090013AE0900795F093
:1032680090013BE0900796F090013CE0900797F0C2
:10327800900090E0900798F0900091E0900799F006
:10328800900092E090079AF0900093E090079BF0EE
:10329800900094E090079CF0900095E090079DF0D6
:1032A800900096E090079EF0900097E090079FF0BE
:1032B800900099E09007A0F090009AE09007A1F0A4
:1032C80090009BE09007A2F090009CE09007A3F08C
:1032D8007400900082F01200C974AB900788F01255
:0A32E80027B674AA900788F0E55895
:063A18000231070231B289
:1032F200903A39F82828738012122861800D122919
:0B3302009F8008122ADD8003122C1BA4
:0F3A39000232F90232FB02330002330502330A74
:10330D00900788E4F090013AE0700C90013BE0707A
:10331D000690013CE060028004C20A8002D20A02DB
:10332D003431C29C900078E0900789F090005EE007
:10333D0090078AF090005FE090078BF090007AE0A4
:10334D0090078CF0900057E090078DF0900062E0B0
:10335D0090078EF0900063E090078FF0900074E07E
:10336D00900790F090007CE0900791F090007DE048
:10337D00900792F0900080E0900793F0900081E02C
:10338D00900794F090013AE0900795F090013BE0A2
:10339D00900796F090013CE0900797F0900090E038
:1033AD00900798F0900091E0900799F0900092E0CE
:1033BD0090079AF0900093E090079BF0900094E0B6
:1033CD0090079CF0900095E090079DF0900096E09E
:1033DD0090079EF0900097E090079FF0900099E085
:1033ED009007A0F090009AE09007A1F090009BE06C
:1033FD009007A2F090009CE09007A3F0740090005D
:10340D0082F074AB900788F01227B674AA900788E3
:10341D00F012286112299F122ADD122C1BD29C75E5
:10342D0099FB80FED29C7514007513007599FB02F3
:10343D00362C900786E0FEA3E0FFEF4E70068599CF
:10344D0010750F00900786E0FEA3E0FF74016F4E2C
:10345D00701BAC0FAD10AA0DAB0EED2BFBEC3AFAB9
:10346D008A068B0790004E12001EE599F090078694
:10347D0012000E900786E0FEA3E0FF74026F4E70FF
:10348D000C1200C985159975140075130002362CA0
:10349D00900786E0FEA3E0FF90004E12001EE59916
:1034AD00F090078612000E900786E0FEA3E0FFACB9
:1034BD000DAD0E8F028E038C068D07903AAD120066
:1034CD002EE493F9740193FEEAD39EEB994009859E
:1034DD00159975140075130002362C900786E0FEC1
:1034ED00A3E0FF90004E12001EE599F090078612A2
:1034FD00000E900786E0FEA3E0FFEFB40006EEB4E9
:10350D000102800302362C90001CE0D394C7400BBF
:10351D0090001CE0C394C8F516801A90001CE0D3EF
:10352D009463400B90001CE0C39464F516800690E4
:10353D00001CE0F516E51675F002A4FFAEF08F6BDA
:10354D00EF90004E124131EFFCE0FDEC9000511276
:10355D004131EDFCE0FDEC2DB51602800302361E67
:10356D000FEF90004E124131E56BFFE0FCEF900044
:10357D0052124131ECFFE0FCEFC39CB51602800303
:10358D0002361EE56B900050124131E56BFFE0FCF9
:10359D00EF900053124131ECFFE0FCEF2CB51671AA
:1035AD00E56B900054124131E0C3951690079DF0E4
:1035BD00E56B900055124131E0C3951690079EF0D2
:1035CD00E56B900058124131E0C3951690079FF0BE
:1035DD00E56B900059124131E0C395169007A0F0AC
:1035ED00E56B90005A124131E0C395169007A1F09A
:1035FD00E56B90005B124131E0C395169007A2F088
:10360D0012272C7599F97518647517001226E88024
:0F361D00FE7599FF7518647517001226E880FE78
:093A1E0002343F02349D0234E839
:10362C0022E513903A27F828287302376D90078605
:10363C00E0FEA3E0FF90001212001EE0F599900747
:10364C008612000E900786E0FEA3E0FF74116F4E09
:10365C00700375130002376D85629902376D900700
:10366C0086E0FEA3E0FF90004E12001EE0F599EFFD
:10367C00B40107EEB4070375130090078612000E11
:07368C0002376D900787E093
:0F3A270002363602363902366402366A02368FAC
:10369300903A48F8282873852499023762852A9935
:1036A30002376285449902376285479902376285FA
:1036B30051990237628560990237628556990237BC
:1036C30062855899023762756E00900069E0700652
:1036D300900068E060028016A2A44006E56E4404F0
:1036E300F56EA2A54006E56E4402F56E801A9000C1
:1036F3004AE0B40106E56E4410F56E900049E0B46B
:103703000106E56E4420F56EA207B34006E56E445C
:1037130001F56EA209B34006E56E4408F56E856EA9
:1037230099803CA210B340077599FAC2108017A282
:103733000CB3400575990F800B900023E0F5999029
:103743000023E4F0C20C80178542998012854B99BF
:0F375300800D85469980087599FC8003751300D9
:103A480002369A0236A00236A60236AC0236B20216
:103A580036B80236BE0236C40236CA0237260237E4
:0D3A68004B02375002375502375A02375FC4
:0B37620090078612000E800312004842
:033A360002376AEA
:10376D002290006BE0B4010385241190006BE0B44E
:10377D000203852A1190006BE0B403038544119078
:10378D00006BE0B4040385471190006BE0B40503B2
:10379D0085511190006BE0B4060385561190006BB6
:1037AD00E0B4070385581190006CE0FE90006DE0C9
:1037BD00C39E500302384490006BE0D39404402C18
:1037CD0090006CE0D39511500990006DE0C39511F8
:1037DD0050028002D20090006CE0D39511500990F8
:1037ED00006DE0C395115002C200804990006BE05E
:1037FD00B4041890006DE0C395115002D2009000F2
:10380D006CE0D395114002C200802A90006CE0C399
:10381D009511500990006DE0D3951150028002D2A0
:10382D000090006CE0D39511500990006DE0C395A8
:10383D00115002C200807E90006BE0D39404402CA6
:10384D0090006CE0C39511400990006DE0D3951187
:10385D0040028002C20090006CE0C39511400990B7
:10386D00006DE0D395114002D200804990006BE0CD
:10387D00B4041890006CE0C395115002C200900082
:10388D006DE0D395114002D200802A90006CE0C308
:10389D009511400990006DE0D395114002D2009032
:1038AD00006CE0D39511400990006DE0C395114077
:1038BD00028002C2002290006EE0B4010385241143
:1038CD0090006EE0B40203852A1190006EE0B403FF
:1038DD000385441190006EE0B404038547119000F8
:1038ED006EE0B4050385511190006EE0B4060385BA
:1038FD00561190006EE0B4070385581190006FE0EB
:10390D00FE900070E0C39E500302399990006EE066
:10391D00D39404402C90006FE0D395115009900082
:10392D0070E0C3951150028002D20290006FE0D377
:10393D0095115009900070E0C395115002C202809C
:10394D004990006EE0B40418900070E0C3951150DA
:10395D0002D20290006FE0D395114002C202802A7C
:10396D0090006FE0C395115009900070E0D3951150
:10397D0050028002D20290006FE0D3951150099051
:10398D000070E0C395115002C202807E90006EE07F
:10399D00D39404402C90006FE0C395114009900022
:1039AD0070E0D3951140028002C20290006FE0C317
:1039BD0095114009900070E0D395114002D202801C
:1039CD004990006EE0B4041890006FE0C39511505B
:1039DD0002C202900070E0D395114002D202802AFB
:1039ED0090006FE0C395114009900070E0D39511E0
:1039FD004002D20290006FE0D39511400990007003
:0B3A0D00E0C3951140028002C20222BB
:094131002582F58250020583226B
:10002E00EF2F500205832582F582E5833E2EF58360
:01003E00229F
:08000300C3EF9DFFEE9CFE22FD
:08003F000806B60002180622B3
:0D000E00A3E004F07006124127E004F02288
:084143000816B6FF021816224F
:0E410B00048007C3CE13CECF13CFD5E0F6222B
:103FB900BC000FBE0008ED8FF084FFADF022E4FED7
:103FC900FF22BE000DEF60FE54F0606F20E7030290
:103FD900406FEAC0E0EBC0E078017A0075F001EECD
:103FE90020E710EF25E0FFEE33FE0AC5F023C5F008
:103FF90030E7F0EA5407F9096A7A007B00600108A2
:10400900C3EC9E40167004ED9F4010ED9FFDEC9EA1
:10401900FCE5F0CA4ACA03F5F08005E5F003F5F0BE
:10402900C3EE13FEEF13FFD9D77908CACBCAD8D08C
:10403900EAFEEBFFD0E0FBD0E0FA22EC8FF084FC43
:10404900ED54F045F0C48FF084FEEDC454F045F012
:10405900C48FF084FDEEC4FE54F02DFFEE540F3CE6
:10406900FEADF07C0022790078008FF0EC7E08200C
:10407900E70DC3CD33CD33C933C9C833C8DEF084A6
:1040890049F9E5F08FF0BE00E6FD7C00E9FFE8FEA6
:014099002204
:0E411900F88FF0A4FFE5F0CE88F0A42EFE2271
:1040EB00600D782B0240F5007830D8FED5E0F82231
:1040FB00EEC0E07E00123FB9EFFDEEFCD0E0FE22F9
:03000B0002409A16
:03001B000240B5EB
:03002B000240D0C0
:0300000002413A80
:09413A0075817275D0000207FDC9
:0B001E00E5822FF582E5833EF583228A
:0A4127000582D5820215831582225D
:10409A00C0E0C0F0C083C082C0D075D0001207F261
:1040AA00D0D0D082D083D0F0D0E032C0E0C0F0C00F
:1040BA0083C082C0D075D0001207F5D0D0D082D08C
:1040CA0083D0F0D0E032C0E0C0F0C083C082C0D05C
:1040DA0075D0001207F8D0D0D082D083D0F0D0E0CB
:0140EA0032A3
:00000001FF
